:020000000125D8
:2000230001D07598D0758920758DFDD28ED2ACD2AFC27F757F63757E01757D01757C0175AD
:200043007B01757AF87579FC7578FE7577FF7F007590F0A87FD8FE857A90A87ED8FE857980
:2000630090A87DD8FE857890A87CD8FE857790A87BD8FE7590F0207F030200567590FFC231
:200083007F11C5B400030200ACF576BF00027F0974809FF9E576F7C2AFEFF59920990280E8
:2000A300FB11DE1FD2AF020056C2AF7E0974809EF9E7F59920990280FB11DEDEF0D2AF02ED
:2000C3000056E59922207EFDF599D27E22309906C299C27E8004C298D27F327A037BFFDBEF
:2000E300FEDAFA222A2A2A2A2034204368616E6E656C2050574D2046616E20436F6E7472C5
:200103006F6C202A2A2A2A2A2A2A10286329203230303320486172647761726520627920A9
:1F01230052756E6E69202D2D2D20536F66747761726520627920656C48616B696D1000B9
:00000001FF
